:100000000C946E00189518951895189518951895D4
:100010001895189518951895189518951895189578
:100020001895189518951895189518951895189568
:100030001895189518951895189518951895189558
:100040001895189518951895189518951895189548
:100050001895189518951895189518951895189538
:100060001895189518951895189518951895189528
:100070001895189518951895189518951895189518
:10008000189518951895189518951895392F482F83
:10009000F894E0E0F0E006C001968A352AE0920785
:1000A000D8F33196E017F10718F480E090E0F5CF2F
:1000B0007894842F932F08958A938EEF0FEF07BBC8
:1000C00008BB88BB880F81608F3F09F48EEF04EF77
:1000D00011E0DCDFF6CF00008895FECF0FE30DBF07
:1000E00001E00EBFC0E2D1E00E947C000E945C00F3
:0C00F0000E946B000C946B0001E008956E
:00000001FF
